:020000020000FC
:10000000F3C98FC20000000025C000004DC10000F0
:10001000000050C1000000000000000002030406C0
:10002000080C101820304060800002030406080C01
:10003000101820304080FF000406080C10182030F3
:10004000406080A0C0000D0D0403060D050D0602E2
:10005000030202004FB662FD1EC070FF18C165FDAD
:10006000F8C00994C0919700C395C0939700C5E06C
:10007000C519B8F3D0919700CD1B98F3C8E7089441
:1000800083FDC795C4BDC52DCC2321F4C0E083FDFD
:10009000C0E8C4BD07C171FF03C0919890989398C0
:1000A000C52D089483FDC795C4BDC09399006B7F8F
:1000B000C52DCF3F09F441C0C0919800C395C093AE
:1000C000980070FF35C09198909893984FBE1895FE
:1000D0007860C091A000CC2391F0C0919800CA959F
:1000E000D091A000CD1B58F0777FC0919800D0919F
:1000F0009F00CD1B08F41CC02092980019C0919855
:1001000090989398C5E0CA95F1F7C0917500CA958B
:10011000C2FD09C0C1FD05C095FF959A95FD949A51
:100120000EC0979A0CC095FF949A95FD959A07C0BA
:100130009198909893984FBE1895209299004FBE31
:100140001895A5C0552021F095FF919A95FD939A99
:1001500090989DC0552009F0909A95FF939895FD31
:10016000919895C0552021F095FF939A95FD919A0D
:1001700095FF919895FD93988AC095FF949895FD69
:10018000959895FF959895FD9498C5E0CA95F1F7D7
:10019000552021F095FF919A95FD939A909877C0FC
:1001A00095FF949895FD95989798C5E0CA95F1F7B5
:1001B000552021F095FF919A95FD939A909867C0EC
:1001C000979895FF949895FD9598C5E0CA95F1F795
:1001D000552009F0909A95FF939895FD919857C0F6
:1001E000979895FF959895FD9498C5E0CA95F1F775
:1001F000552009F0909A95FF939895FD919847C0E6
:1002000095FF959895FD94989798C5E0CA95F1F754
:10021000552021F095FF939A95FD919A95FF91981D
:1002200095FD939834C095FF959895FD949895FF0A
:10023000949895FD9598C5E0CA95F1F7552021F061
:1002400095FF939A95FD919A95FF919895FD9398B6
:100250001EC082FF1CC0C0917500C2FD0BC0C1FD55
:1002600011C095FF949895FD959895FF959895FDEB
:1002700094980DC0C1FDF5CF95FF949895FD959884
:10028000979805C0979895FF959895FD9498C52DDA
:10029000C095089483FDC795C4BDC0939900209272
:1002A000970064604FBE18954FB6C0E1C8BF6E7F1F
:1002B0004FBE18953FB68F7EABB7A074A211806178
:1002C000A0E0ABBFA9B7AE7FA9BF7894A0916600AC
:1002D000AA2349F0A92FAF7151F1A0916600AA9508
:1002E000A093660024C040E050E0A0B396FFA09524
:1002F000A2FD4FEF96FDA3E096FFA2E0A5BFAA27BF
:10030000A064AABF8D7FA0B396FFA095A2FD5FEF6A
:10031000451749F7A0E461FDA0936600A92FAF71CE
:1003200019F0A0E4A093660040938D008160A09135
:100330006700AA2331F0A0916700AA95A0936700F7
:1003400007C0A92FAF7121F08061AA27A064AABFBE
:1003500080FF30C0A0918D004A2F8E7FA92FAF71F2
:1003600009F000C04093610071FF08C0A0916100D6
:1003700050919200A51710F0509361004091AE008B
:100380004430C1F4A091610040916300A41B70F05F
:100390004091CF00A40B50F0A0916300A40FA09354
:1003A000630040F4AFEFA093630004C0A09161002C
:1003B000A0936300A52DA03408F06860A0916000B0
:1003C000A395A093600051F0F894A9B7A160A9BFCC
:1003D00084FF02C0A0E4ABBF3FBE189542E050913D
:1003E0006600552331F0A92FAF7119F45A95509337
:1003F0006600A0918D00A13018F0209290000DC0F1
:100400002092910020929A00A0919000AF5FA0935B
:10041000900018F0AFEFA0939000B0906100509161
:10042000AE00523049F466FF91F0A2E3BA1678F0BC
:10043000A0917F00A0936100533049F466FF39F02A
:10044000A2E3BA1620F0A091BA00A09361005091E7
:1004500062005B1521F010F05A9501C0539550933E
:1004600062004A95D1F650919A00539509F45A9535
:1004700050939A00A0919B00AA95A0939B0009F02D
:1004800046C0A1E0A0939B0045E0A0919C005A17B4
:10049000F0F1A0919D005A1728F441E0A3E0A09349
:1004A0009B0007C0A0919E005A1718F441E04093AA
:1004B0009B00D0909300C0906300DC14A8F0A09142
:1004C000AE00A430D9F066FD0FC0C09293005395E2
:1004D00019F0A0919C00A0939A00A1E0A0939B002A
:1004E000ACE3A093620013C0A0919300A40F20F48A
:1004F0005FEF5093930002C0A0939300A0919300EC
:10050000AF3F29F4AFEFA0939100A0939A00F89425
:10051000A9B7A160A9BF84FF02C0A0E4ABBF3FBEE2
:1005200018953FB64CB55DB58F7EABB7A074A211E0
:100530008061A0E0ABBFA9B7AE7FA9BF789481FD71
:1005400026C096FDA2E096FFA3E0A5BF8260A0B3FF
:1005500096FFA095A2FF05C04093640050936500EC
:10056000FDC096FDA3E096FFA2E0A5BFAA27A06468
:10057000AABF8D7FA92FAF7109F4E1C040E0A0B3FD
:1005800096FFA095A2FDDBC040938D00CEC096FDE6
:10059000A3E096FFA2E0A5BF8D7F61FF6BC096FD33
:1005A000A2E096FFA3E0A5BFAA27A064AABF82602D
:1005B0004093880050938900A09086004A19B0901B
:1005C00087005B09BB24A2E0EA2EA22C483CA0E0F5
:1005D0005A0730F4A0E1BA2EE22CAAE0AA2E27C0D6
:1005E0004836A1E05A0730F4A8E0BA2EE22CAFE07A
:1005F000AA2E1DC0403DA2E05A0730F4A4E0BA2E56
:10060000E22CAEE1AA2E13C0403AA5E05A0730F41E
:10061000A2E0BA2EE22CACE3AA2E09C04839A8E029
:100620005A0728F4A1E0BA2EE22CA8E7AA2EC42E7D
:10063000A0918A00CA1AD52EA0918B00DA0ADD207B
:100640002AF4AFEFC094D094CA1ADA0A20928C0030
:10065000CA14DE0418F4A1E0A0938C0040938A0031
:1006600050938B0040918800509189004093860000
:1006700050938700A09164004A1BA09165005A0B1B
:1006800094FD46C093FD44C092FD40C056954795E9
:1006900091FD3CC05695479590FD38C0D52EC42E8F
:1006A000D694C79461FD0CC0AC2DAC51AD2DA240C9
:1006B00008F045C0DD2021F4AC2DA85C08F43FC053
:1006C000A0E0EA2E97FD02C0E090C200AAEFEA0E79
:1006D000F22CF21CCE18DF084FB74170442319F0FA
:1006E00040E050E015C0AFEFCA16D20418F04FEF4B
:1006F00050E00EC0F090A700CF9C412D000C441F8D
:1007000050E008F012C04FEF50E00FC056954795EB
:1007100094FF07C0552309F04FEFA42FA6954A0F69
:10072000521D4F3F520508F04FEF40938D008160FE
:1007300061FF05C0AFE1A095A923AB299A2FA0E4E2
:10074000A0936600A92FAF7119F4AAE0A0936600E8
:1007500061FD04C0A92FAF7109F08F7EA0E2A093C4
:100760006700A92FAF7119F4AAE0A0936700F8946D
:10077000A9B7A160A9BF84FF02C0A0E4ABBF3FBE80
:10078000189511E00AC013E008C01AE006C01EE187
:1007900004C014E602C018EC00C005E1BB27BA95FE
:1007A000F1F70A95D9F71A95C1F708952AE338E7C2
:1007B00009C020E33CE806C02AE234EB03C025E28E
:1007C00038EC00C0652CB1E05B2E12E095FD9F7DFA
:1007D00095FF9062BB279798BA95F1F7552009F0DD
:1007E000909ABA95F1F79098BA95F1F7979ABA95C9
:1007F000F1F7552021F095FF919A95FD939AB091CC
:10080000A800BA95F1F795FF919895FD9398B7E8F0
:10081000BA95F1F71A95D1F6022FB22FBA95F1F7E2
:100820000A95D9F73A9571F69798562C0895221B98
:1008300039E0001F3A9509F40895221F211B18F48E
:10084000210F8894F6CF0894F4CF622C722CB0E07C
:100850008894B395221F331FE0F737952795889426
:10086000912E802E020B130B10F4192D082D10F46D
:10087000889401C00894661C771CBA9571F7172DEF
:10088000062D0895322D11232AF43A9500951095DE
:10089000031B130BF894029F712C002D129F912CB7
:1008A000802C7894780C172D921C292DB4E06B2E97
:1008B0002695179507956A94D9F7332321F000956B
:1008C0001095031B130B08950091AE00043009F43A
:1008D00074C0B0918D00B95198F0B72FB67081F403
:1008E00066FD2BC005E09090C000B92DBA9521F0AF
:1008F0000AE0BA9509F002E1B0917400B01BE0F093
:1009000066FF0AC0B0919500B0939300BFEFB0931B
:100910009A00B1E0B0939B00B0916100B093630086
:1009200020927700209278002092790020927A001D
:1009300020927B006F7B41C060649090C000B92D15
:10094000BA9579F4B0916200B095BB1FBB1F1B2F05
:10095000B7950B2FB12FB170B3951B2FB02FBE7F62
:1009600025C0B92DBA95BA9581F4B0916200B095C1
:10097000BB1FBB1FBB1F1B2FB7950B2FB12FB37016
:10098000B3951B2FB02FBC7F14C0B0916200B095FF
:10099000BB1FBB1FBB1FBB1F1B2FB7950B2FB12F3F
:1009A000B770B395B3951B2FB02FB87FB0540B2FF2
:1009B00012090093770010937800089566FF21C014
:1009C000109174001695009173000795B09177000F
:1009D000B01B0B2FB0917800B10B1B2F28F40038FF
:1009E000BFEF1B0740F009C00F37120508F405C020
:1009F0000FE710E002C000E81FEF00937C001093A7
:100A00007D00089566FF39C000917C00B0917900A7
:100A10000B0F10917D00B0917A001B1F20E03091E8
:100A20007D0033230AF42A95B0917B002B1F1AF422
:100A3000203F40F00AC02F3008F407C00FEF1FEF2F
:100A40002FE003C000E010E020EF30916300B09190
:100A500092003B1718F4332331F009C0B0917D00A8
:100A6000BB235AF004C0B0917D00BB2332F4009345
:100A7000790010937A0020937B00089566FF2FC0C1
:100A80002091CD0000917C00000F10917D00111F7E
:100A9000F9DE11232AF40038BFEF1B0740F009C02C
:100AA0000F37120508F405C00FE710E002C000E898
:100AB0001FEF002352F0B0916200B01B0B2F18F013
:100AC000013008F00AC001E008C000950F5FB09146
:100AD00062000B0F08F001C00FEF00937E00089535
:100AE00066FF2DC02091CE0000917A0010917B000E
:100AF000C9DE11232AF40130BFEF1B0740F009C003
:100B00000F3F120508F405C00FEF10E002C001E02E
:100B10001FEF112352F0B0917E00B01B0B2F18F085
:100B2000013008F00AC000E008C000950F5FB091E6
:100B30007E000B0F08F001C00FEF009363000895D3
:100B40000FEF677FB72FB670E9F46860B09174005B
:100B5000B83008F0677FB0917400A1F00FEF1091EA
:100B6000740065DEF894B09170000B9F112D002D7C
:100B70007894112309F00FEFB09195000B1710F442
:100B8000009195000093940008950AD374FFB7E094
:100B900074FDB7E0B068B064B7B9B6B1B068B0641E
:100BA000B6B9EFDD74FFB7E074FDB7E0B068B064CC
:100BB000B7B9B6B1B068B064B6B9B6B1B6FDFDCFDD
:100BC00004B115B1B6B1BF77B6B923D32DE62093E2
:100BD000A30030E03093A400732E7694622E6694C6
:100BE000620E731E262D372D0217130778F08090A2
:100BF000A300BDE6B80DB093A3008090A400B0E0C0
:100C0000B81DB093A400260D371DEECF8090A30031
:100C10009090A4001091A40016950091A300079550
:100C200016950795B091A300B00FB093A100B091B5
:100C3000A400B11FB093A20023E0169507952A9552
:100C4000E1F72091AF002A9529F42092A300209289
:100C5000A4000AC02A9521F0800E911E2A95E1F782
:100C60008092A3009092A40008952091AF00B6B1A5
:100C7000B6FDFBCF04B115B1B6B1BF77B6B9B0912F
:100C8000A500B395B093A500B83060F12092A500FF
:100C9000B091CC00BB2321F1112329F0B091A60023
:100CA000BF3F61F009C0B091A6000B1739F020F4E6
:100CB000BB2321F0BA9502C0B395E1F300919200F5
:100CC000B093A600B03050F400ECB03038F400E837
:100CD000B03020F400E4B03008F400E0009392005B
:100CE0007F7E0895213099F00F3FB3E01B0778F421
:100CF000B091A3000B17B091A4001B0740F4B09172
:100D00009200BB2359F0BA95B093920007C0B091FE
:100D10009200BF3F19F0B395B093920000919200FA
:100D2000B0916300B01B10F400916300B091930088
:100D30000B1750F000919300B0919300BF3F21F04A
:100D4000B0919300B0939200502EB091A500B730AF
:100D500009F47061089502E3F894B091D0000B9FFC
:100D6000012D000C001F7894B09192000B1710F029
:100D7000009192000093610000936300502E009355
:100D80009500089520927300B8E0B0937400089520
:100D90002091800030918100F8940CB51DB5200F92
:100DA000311F3BBD2ABD6160B0E1B8BF789420918E
:100DB0007100309172000093710010937200021B59
:100DC000130B2091730030917400622E732EB4E0E7
:100DD0008B2EB2E09B2EB0917400B43010F08A9448
:100DE0009A94B83010F08A949A94769467948A947E
:100DF000E1F726193709992021F0169507959A945D
:100E0000E1F7200F311F209373003093740008F036
:100E10000895BFEFB0937300B093740008952091CC
:100E2000820030918300F8940CB51DB5020F131F9A
:100E30001BBD0ABD6160B0E1B8BF7894089560FD44
:100E4000FECFEDDF0895B091BE0000916E00023834
:100E500008F0B395003A08F0B395B63008F0B5E065
:100E60009B2EBCE08B2EB0917400B33030F4839491
:100E7000839482FF02C083948394B23030F48394CD
:100E8000839482FF02C08394839471FF03C0B3E014
:100E90009B2E822C109174000091730024E0169513
:100EA00007952A95E1F70819120928F0B02FB250DA
:100EB000B12FB20910F402E010E0312F202F712E73
:100EC000602E76946794B92DB330E9F0B0FD05C07B
:100ED000060D171D262D372D06C0000F111F0250BD
:100EE000120922E030E0B92DB33068F0209384007D
:100EF00030938500009380001093810060928200FF
:100F000070928300089500938400109385002093CD
:100F10008000309381006092820070928300089577
:100F200060FDFECF20918200220F30918300331F9D
:100F3000B72FB67021F02091730030917400F894AF
:100F40000CB51DB5020F131F1BBD0ABD6160B0E1DA
:100F5000B8BF7894089560612092760020E004C0C4
:100F600060612092760020E2B72FB67009F06F7EA4
:100F7000789460FD05C0B0917600BB2309F0089518
:100F800001E063FF0AC0B0917400B33008F002E0E2
:100F9000B0917400B63008F003E071FF01C006E0C4
:100FA00060FD06C0B0917600BB2311F078940895DF
:100FB0001AE083FF1AE0789400000000F89462FDC4
:100FC00003C014E183FF14E171FF01C018E7B4B559
:100FD00030919900B31BB10B18F3B0917600B39523
:100FE000B0937600B5E03B2F6B2E722CB8B1B07287
:100FF000B21709F073943A95C9F77394761488F48C
:1010000064FFB2CF6F7E3CB56DB47090730080907A
:101010007400370D681C6BBC3ABD6160B0E1B8BFAD
:10102000A3CF64FDA1CF0A9509F0BACF78940895B3
:1010300071FF0AC0B0916D00B395B0936D0060FD73
:101040000CC020926D0009C060FD07C064FD05C0A2
:1010500067FD03C0BF91BF916DC4089520918400C6
:1010600030918500F8940CB51DB5020F131F1BBD00
:101070000ABD6160B0E1B8BF78940895EFDF00E089
:1010800063FF03C064FF01C001E0F89410916E009B
:10109000B7E01B9F212D102D7894200F26951795D2
:1010A000269517952695179510936E00183718F406
:1010B000B8E7B0936E0000916E00B0916F000B170F
:1010C00020F0606291989098939860FDFECF08950B
:1010D000F89494989798959882FF07C0E0E0F1E023
:1010E00073FF03C0BEE1BA95F1F795FF949A95FDA1
:1010F000959AB2E0B093750089C0F89495FF9398E3
:1011000095FD919882FF0DC0E0EFF0E073FF0BC0FA
:10111000979895FF959895FD9498BEE1BA95F1F74B
:1011200002C0EAEAF0E062FF03C0552009F0909A9D
:10113000B3E0B09375006AC0F89494989798959826
:1011400082FF07C0E0EEF0E073FF03C0BEE1BA9596
:10115000F1F795FF959A95FD949AB4E0B0937500D8
:1011600055C0F894909882FF0DC0E0EDF0E073FF59
:101170000BC095FF949895FD95989798BEE1BA9508
:10118000F1F702C0E2EAF0E062FF06C0552021F06C
:1011900095FF919A95FD939AB5E0B093750036C08E
:1011A000F89494989798959882FF07C0EDEBF0E03B
:1011B00073FF03C0BEE1BA95F1F7979AB6E0B0931A
:1011C000750024C0F89495FF919895FD939882FF3F
:1011D00010C0E3E1F1E073FF0EC095FF949895FD18
:1011E000959895FF959895FD9498BEE1BA95F1F77D
:1011F00002C0E2EBF0E062FF06C0552021F095FF4F
:10120000939A95FD919AB1E0B09375006F7D7894B3
:10121000089521EA30E0F901919890989398949874
:10122000979895986B7F0895ACEAB0E007E00D932E
:1012300007E00D9301E00D9304E00D930FEF0D9384
:101240000D930AE00D9302E00D9301E00D9301E090
:101250000D93A8EBB0E001E00D9300E00D9304EBDB
:101260000D930FEF0D930D930D9303E00D9301E09C
:101270000D9301E00D930FEF0D9305E20D9300ED3B
:101280000D9308E70D9308EC0D9304E00D930DE02A
:101290000D9301E00D9300E00D930AE70D930AE032
:1012A0000D9301E00D9308952091BF0009E011E036
:1012B000223011F405E011E0233011F405E012E0D2
:1012C000243011F405E013E0253011F409E017E0B3
:1012D000263011F400E010E000939F001093A0006E
:1012E0002091B3008B7F777FB091B4009F7DB1FDDB
:1012F00090629F7BB091B500B1FD9064B22FB23087
:1013000011F0886001C0877F0895ECE1F0E0009162
:10131000AC000A95E00FF21DB491B093CD0000919E
:10132000AD000A95E00FF21DB491B093CE0071DFCD
:101330000895EAE2F0E00091C7000A95E00FF21D7F
:10134000B491B093CF0065DF0895E8E3F0E0009139
:10135000B2000A95E00FF21DB491B093D00059DFAE
:1013600008950091CB00002309F40395013108F0A2
:1013700001E1B02FB00FB00FB0939C001B2FB10F45
:10138000B10FB00FB0939D00B10FB00FB00FB0937D
:101390009E000895B091C8000FEF1CE0B23011F428
:1013A00000EA1AE0B33011F402E815E000936F0090
:1013B00010937000089508952091C2003091C300E9
:1013C00097FF02C020E03FEFB32FB21B6B2EB25845
:1013D00010F4B2E86B2E00E00395609EB12DB0587A
:1013E000D8F30093A7000895F894E3E0F0E0B9E0A3
:1013F000B7BFB491B078C1F3F894A895B1B5B8610E
:10140000B1BDB0E0B1BDB4E0BEBFBFE5BDBF01DF5F
:10141000B0E0B8BBB0E1B7BBB0E0B5BBB0E0B4BBC7
:10142000B0E0B2BBBBEBB1BB2224A0E0B0E02D9298
:10143000AA31E9F7A0E6B0E00FEF2D920A95E9F79F
:10144000F3DE9DD231DF61DF74DF7FDF8ADFA2DF71
:10145000B2DFB2DF0091C4000093A800DADEB2E090
:10146000B3BFB2E0BEBDB2E0B5BDF89494D99ED989
:101470008ED99FD98CD9A0D98AD918D38CD98BD998
:1014800088D9B1E5B8BFB9BFB0B7B860B0BFB6B121
:10149000B460B6B976D9789478DBB0E4BBBFBB272B
:1014A000B064BABF8D7F77D9B1E0B0936900626054
:1014B00025E0B0918C00BB2309F425E064D9B091FC
:1014C0008D00B230A8F3B92FBF7100918F00009347
:1014D0008E00B0938F00B01759F72A9551F76D7FA2
:1014E00096FDB3E096FFB2E0B5BFBB27B064BABFCC
:1014F0008D7F4FD948D902E0B92FBF7109F400E0C0
:10150000B0918D00B017B0F3F89450D94FD94ED99F
:10151000789441D920927F0036D9B091B800B1308B
:1015200008F46CC0B0916900B13008F467C0B92FFD
:10153000BF71C1F0B0918D00BF3F08F45FC0F89457
:101540003ED9789426D9B0918D00B130C0F7F89487
:101550002DD91BD92BD978941CD9B0918D00BF3FC0
:10156000B0F3D6C2B8E09B2E9068F89425DF78944B
:1015700010D9F8949F7720DF80908D00B0918D0076
:10158000BF37789408F442C0FCD8F89418D97894FE
:101590009A9451F7B82DB550B093C300FCD8F89485
:1015A0001BD289D27894BAE09B2E9068F89404DF1D
:1015B0007894EFD8F8949F77FFDE80908D00B091FB
:1015C0008D00BF37789478F7DCD8F894EFD8DDD861
:1015D000EDD878949A9449F7B82DBB5FB093C200C8
:1015E000DAD8F894F9D176D27894D3D8F894E4DEA6
:1015F0007894B0918D00BF3FC0F38AC200918D00F6
:10160000B0917F000B1710F000937F00C2D801E06B
:10161000B091B400B35009F405E0B0918D00B0175B
:1016200008F07ACFF894CBD8CAD8C9D87894B3D870
:101630002092690020926A0020926B00B0916A00AB
:10164000B395B0936A00BF3F69F5B0916B00B39555
:10165000B0936B00B091C60009E1BA9559F002E36E
:10166000BA9541F00DE7BA9529F00AEFBA9511F055
:1016700020926B00B0916B00B017A0F0B0916B009E
:10168000BA95B0936B00B4EBB0936A00B091C5000B
:10169000B093A800F89493D87894B091C400B09314
:1016A000A80077D872D8B0916600BB2321F4B92F77
:1016B000BF7109F4FCCEB0918D00B63008F4BECFF6
:1016C00068D8B0916600BB2309F4F1CEF894A1DD8F
:1016D000209261002092620020926300522C789444
:1016E000B091B100B09396002092770020927800DC
:1016F0002092790020927A0020927B002092A5000F
:1017000060E070E020926E003DDBB8E0B093A50091
:10171000706137D874FFB7E074FDB7E0B068B064AB
:10172000B7B9B6B1B068B064B6B9B6B1B6FDFDCF61
:1017300004B115B1B6B1BF77B6B9112309F00FEFF7
:101740000093A60092DAB8E0B093A5007061809093
:10175000B300B2E0B093B300A7DD8092B300F89479
:10176000BFEFB0939200F7DAB0916100B0939200AE
:10177000B0939300B09394007894B1E0B09361007B
:10178000B09363005B2EB0939B00B0919100B09337
:101790009A007160726020926D0002DD13DDF8DA4C
:1017A000F1DA51DB04C080DD2092A5007F7E95FF39
:1017B000B2E095FDB4E0B068B064B7B9D1DB38DC15
:1017C0004DDC82D85BDC84DCE3DA39DB3CDBA8DB94
:1017D000B3E0B068B064B7B9BEDB2ADC3FDCEED85A
:1017E000AFD94CDC8ADCD4DA2ADB2DDB99DB95FF20
:1017F000B4E095FDB2E0B068B064B7B9B1DB18DC15
:101800002DDC00D93BDC98DCC3DA19DB1CDB88DB80
:1018100095FFB2E095FDB4E0B068B064B7B99BDB6A
:1018200007DC1CDC2BD92ADC9CDCB2DA08DB0BDB06
:1018300077DBB3E0B068B064B7B992DBF9DB0EDCFC
:101840004FD91CDCADDCA4DAFADAFDDA69DB95FFEE
:10185000B4E095FDB2E0B068B064B7B97CDB74FF6A
:10186000B7E074FDB7E0B068B064B7B9B6B1B068BE
:10187000B064B6B9DDDBF2DB01DCA4DC89DADFDAE7
:10188000E2DAF3D94DDB71FF20C067FD1EC0B091D5
:101890009500B0939200B0939300B0919100B093F3
:1018A0009A00B1E0B0939B0014E624E1B0916D0082
:1018B000B11728F07D7F746020936C0006C0B09152
:1018C0008D00B13008F073CF35C072FF10C067FDD6
:1018D0000EC0B0916C00BA9511F47B7F64CFB093C9
:1018E0006C00B0918D00B13008F061CF23C0B09191
:1018F0009000B13058F0B0919500B0939300B09142
:101900009100B0939A00B1E0B0939B00B091900029
:10191000BA3F80F4B92FBF7121F4B0916600BB23A8
:1019200049F0B091740000EF67FF01C000E6B01706
:1019300008F43DCFF8946DDC8090B300B2E0B09332
:10194000B300B2DC8092B30020926100209262006A
:1019500020926300522C209296007E7F789411D7BB
:1019600058DCB92FBF7129F4B0916600BB2309F48C
:101970009ECDB091B900B13008F0BCCD5BCEEDE0AA
:10198000F0E023D0053A09F01BC0EEE0F0E01DD0F6
:101990000A3509F015C03AE0ACEAB0E0E3E0F0E067
:1019A00014D00D9331963A95D9F735E1A8EBB0E014
:1019B000EFE0F0E00AD00D9331963A95D9F702C0E6
:1019C00033DC0AD0E4E2F0E00895E199FECFEEBB0B
:1019D000FFBBE09A0DB308951ED03AE0ACEAB0E048
:1019E000E3E0F0E00D910FD031963A95D9F735E16B
:1019F000A8EBB0E0EFE0F0E00D9105D031963A951C
:101A0000D9F712D00895E199FECF0DBBEEBBFFBB15
:101A1000E29AE19A0895EDE0F0E00FEFF4DFEEE0F6
:101A2000F0E00FEFF0DF0895EDE0F0E005EAEBDF26
:101A3000EEE0F0E00AE5E7DF08953091A9000091BB
:101A4000AA00313011F40093AC00323011F400934D
:101A5000AD00333011F40093AE00343011F4009334
:101A6000C000353011F40093AF00363011F400930C
:101A7000B200373011F40093BE00383011F40093F7
:101A8000C700393011F40093BF003A3011F40093CD
:101A9000B3003B3011F40093C8003C3011F40093C4
:101AA000B4003D3011F40093B500089525E073D6DD
:101AB0002A95E9F708957AD67CD67ED680D665D663
:101AC00075D677D679D67BD660D670D672D674D6D0
:101AD00076D6089574D670D66CD668D656D66FD69C
:101AE0006BD667D663D651D66AD666D662D65ED630
:101AF00008958090A9009090AA0058D657D656D63F
:101B000044D68A94D1F75BD640D69A94E1F70895EB
:101B1000F894D1DF7894CADFC9DFB1E0B093A900AF
:101B2000B1E0B093AA002092AB00F894E2DF789481
:101B3000B5E06B2E70908D002ED6B0918D007B1687
:101B4000C9F7B13018F0BF3F40F107C076DFF89415
:101B500043DFB1DFB8E0B1BDA9DF6A9459F7B091B6
:101B6000AB00B395B093AB00B33008F4DECF9EDF8B
:101B7000B091AA00B395B093AA00F894B091A900CF
:101B8000BA95E6E4F0E0EB0FF21D0491789403952A
:101B9000B091AA00B01708F4C6CF88DF87DFB091F4
:101BA000A900B395B093A900B091A900BE3008F484
:0E1BB000B7CF3ADBF89410DFB8E0B1BD77DFB5
:00000001FF
